:1000000000308A0044280000831605118312051170
:1000100093011308073C031C2A281308073C94008B
:1000200012088C0014088D0003191A2803108C0C78
:100030008D0B16280C181E2885101F288514831672
:100040008510051083120510831605108312051400
:10005000930A0928831605118312051500341130FF
:10006000840000080319432801308D008C018C0B9B
:1000700037288D0B36284A308C008C0B3D28000029
:100080000000800B3428003484011F3083058F0169
:10009000013092000420013090008F010F08073CCE
:1000A000031C5C281008920004200310900D3230CD
:1000B00091002F208F0A4E28803090008F010F086A
:1000C000073C031C6D281008920004200310900CBC
:1000D000323091002F208F0A5F284B280F089100A3
:1000E0009109110892000420643091002F208F0A9A
:0400F0006E28630013
:02400E00F93F78
:00000001FF
